:040000008A15282D08
:08000800FF00030E8312031335
:10001000DD000A0EDE00040EDF008A150A12A22D92
:10002000B408031D14280800A330000000000000DD
:100030000000FF3E031D1528000000000000000026
:10004000B40B1428080083160313DA014030DB00D8
:10005000AA08031D2D280130DA00DA08031D432801
:100060002A08033A031D3628DB0143287F30DB00D2
:10007000B008031940282A08023A0319DB01432873
:100080002A030319DB01831255088316E200831249
:1000900056088316E300831257088316E400831280
:1000A00058088316E5005B08E600E701E801E9016E
:1000B000DB1F5D28E703E803E9036608E20767083A
:1000C0000318670FE30768080318680FE407690857
:1000D0000318690FE5077F30831255058316E0008A
:1000E00000307502031D7628FD307402031C0F29B1
:1000F0007408FD3C75080318031DF51B802888282B
:10010000FD30740603197508031DA128E51FA128F9
:100110002830AB04DB08031D98287F308312D700FA
:10012000FF30D500D600D801FE30F400F5010800FC
:10013000FF30F400F5018312D501D601D701D801B3
:100140000800F51F0F29E70129030319E70AE60153
:100150007508803AEB007F306B02031DB128FF3039
:100160007402031CE60AEA01E6080319E708031D06
:10017000EA0A80306505E800E901E90AE808031D9C
:100180006910E101E9080319EA08031DE10AF4080E
:100190000319F508031901297409E6007509E70038
:1001A000E60A0319E70A2030660267080318DA280E
:1001B0000319DC28E71FF42868107409E900E90A2C
:1001C0008312551CE5288316681403108312D80C7B
:1001D000D70CD60CD50C8316E903031DE028681C48
:1001E0000129831255140129831255085604570416
:1001F0005804FF39031901290130D500D601D70170
:10020000D801F401F5017F30831255058316E00013
:10021000E10803190F29E00803190F292B16E0083C
:10022000031DAB165B08E600E701E801E901DB1FEF
:100230001C29E703E803E90366088312D507831640
:100240006708031C2629670F262928298312D60749
:1002500083166808031C2F29680F2F293129831260
:10026000D70783166908031C3829690F38293A29EA
:100270008312D80707308316E600E60803194929D8
:1002800003108312D80CD70CD60CD50C8316E603BA
:100290003D2940306006031D5229DA08031952290E
:1002A0008312551083125508560457045804FF3919
:1002B000031D0800F401F501080083120313581C04
:1002C00065290230F4070318F50AD71F6B29F40AD1
:1002D000031D6B29F50A7408D8000310D80CD71336
:1002E0007418D7178316B008031908008312D8179B
:1002F0000800403083160313D800E001E101E20159
:10030000E3018312D501D601D701D801831658081D
:10031000D900D803D9080319E82903108312D50D91
:10032000D60DD70DD80D8316E31F982983125514C7
:1003300003108316E00DE10DE20DE30D8312D41FCF
:10034000DF294D088316E00783124E08031CAB29F2
:100350004E0FAB29AD298316E10783124F08031C0A
:10036000B4294F0FB429B6298316E2078312500827
:10037000031CBD29500FBD29BF298316E307831233
:10038000500883166302031DD52983124F08831674
:100390006202031DD52983124E0883166102031DD4
:1003A000D52983124D08831660020318DF298312B2
:1003B000D50A0319D60A0319D70A0319D80A8312D2
:1003C000D81BE8290310D10DD20DD30DD40D8629E9
:1003D000F501203083165802F400031CF503D81BE6
:1003E000F5036008610462046304FF39031908001F
:1003F00083125514080083120317A101A201A3015F
:10040000A40183160313EC01ED01EE01EF01831249
:100410000317A001A01A0800031083160313EC0DA4
:10042000ED0DEE0DEF0DE40DE50DE60DE70D83127C
:100430000317A10DA20DA30DA40D831603136B08C2
:10044000831203172402031D3B2A831603136A0831
:10045000831203172302031D3B2A83160313690823
:10046000831203172202031D3B2A83160313680815
:10047000831203172102031C672A831603136808DB
:1004800083120317A10283160313690803184B2A6A
:10049000690F4B2A4E2A83120317A20283160313F5
:1004A0006A080318562A6A0F562A592A8312031714
:1004B000A302831603136B080318612A6B0F612ACA
:1004C000642A83120317A402831603136C14831285
:1004D0000317A00A0A2AE601E701E6190800651CCD
:1004E000732A6408E707E50C0310E40DE60A6D2A99
:1004F000BC01BF01C0013208BD003308BE003C1A78
:100500000800341C892A3D08BF073E0803183E0F27
:10051000C0070310B50CB40C0310BD0DBE0DBC0A12
:100520007F2AEC01ED01EE01EF0183120317A10117
:10053000A201A301A401A001A01A08000310A10DAB
:10054000A20DA30DA40D83160313E80DE90DEA0D0A
:10055000EB0DEC0DED0DEE0DEF0D63086F02031DBD
:10056000BB2A62086E02031DBB2A61086D02031DCF
:10057000BB2A60086C02031CCE2A6008EC026108EA
:10058000031C610FED026208031C620FEE02630898
:10059000031C630FEF028312031721148312031746
:1005A000A00A9C2A831285118316CC0110304C02BC
:1005B0000318012B4A08D1004B08D2004C08FF3920
:1005C0000319E72A0310D10DD20DFF3EDF2A51088F
:1005D000CD005208CE0000304D05CF004E088039C6
:1005E000D000CF08031DF72AD0080319FA2A831276
:1005F0008514FC2A83128510051505118316CC0A73
:10060000D62A831285150800831203135508560451
:1006100057045804FF390319192B581B08000310FD
:10062000D50DD60DD70DD80DF4080319F503F40335
:100630000D2BF401F5010800D901D70183134D18E2
:1006400083174C0884005708D70A84070008D8008D
:10065000D8080319762C5808253A031D3C2B831320
:100660004D1883174C0884005708D70A84070008E0
:10067000D800253A031D472B83134B1883174A08CC
:1006800084005908D90A8407580880001E2BDB0112
:100690005C102030DA005808003A0319762C303A02
:1006A00003195C2B103A03195F2B0B3A0319622BC9
:1006B000063A0319652B712B3030DA00662B203097
:1006C000DB00662B2B30DB00662B5C1483134D188C
:1006D00083174C0884005708D70A84070008D800FD
:1006E0004B2BDD0130305802031C932B5808393C4A
:1006F000031C932B5D08E4000A30E5006B226708B9
:10070000DD005808DD073030DD0283134D188317F4
:100710004C0884005708D70A84070008D800D80876
:100720000319762C722B58086F3A0319A72B0B3A32
:100730000319AA2B083A0319AA2B193A0319B92B42
:100740002D3A0319BC2B3A3A0319BF2B762C0830EB
:10075000E000C12BD61FB92B2D30DB00D309D40903
:10076000D509D609D30FB92BD40FB92BD50FB92B77
:10077000D60A0A30E000C12B1030E000C12B023055
:10078000E000DE015308E4005408E5005508E600E7
:100790005608E700DE0A6408E8006508E900660814
:1007A000EA006708EB006008E000E101E201E30114
:1007B0009122210883160313E400831203172208F1
:1007C00083160313E500831203172308831603130C
:1007D000E60083120317240883160313E700640856
:1007E000650466046704FF39031DCA2BDB08031D7B
:1007F000DE0ADF015D08003C0318082C5E085D027C
:100800000318042C5D08DE005E085D02DF000B2C7F
:100810005E08DD00DF01DF0803195C105D08D90701
:10082000DC105C18DC14DE08031D192CDF0803192A
:10083000732CD903DC1C222C5A08D800DF0B6A2C3D
:10084000DC106A2CDE0B2A2CDB0803192A2C5B082F
:10085000D800672C5308E4005408E5005508E6006A
:100860005608E7006008E800E901EA01EB01FB2116
:10087000210883160313D8005808093C0318432C99
:100880003730D807452C3030D8075308E8005408D3
:10089000E9005508EA005608EB00E101E201E30136
:1008A0009122210883160313D30083120317220811
:1008B00083160313D400831203172308831603132C
:1008C000D50083120317240883160313D600DE080D
:1008D0000319DC1483134B1883174A085907840043
:1008E00058088000132C5D08D9071E2B83134B1862
:1008F00083174A08590784000030800008004E081A
:100900008312CD0083164F088312CE008316500841
:100910008312CF00CF13D00183165108AC00AC1363
:100920000310AC0DD01B2C14AE01D11F992C01303B
:10093000AE00D30196302C02D200031CD3038030CA
:100940002C02D4005408153C03183A2DD41B3A2D20
:1009500054081D3C0318DF2CD41BDF2C4E08003C30
:10096000031DBE2C4F08003C031DBE2C5008003C4C
:10097000031DBE2C5108CF3C0319D82C2B14AE08F4
:100980000319D02C54087F3AD41BD82C031DD82C23
:1009900083124D084E044F045004FF390319D82C1C
:1009A0007F308316DC00FF30D900DA00DB0008005E
:1009B0008316D901DA01DB018030DC000800163033
:1009C000D4028312CF1783165408DD00DD08031903
:1009D000F22C03108312CD0DCE0DCF0DD00D83164A
:1009E000DD03E62CAE080319292D83124D08003CC7
:1009F0008316DD000030DE00DF00E00083124E08C9
:100A00000318052D4E0F052D072D8316DE028312C8
:100A10004F0803180E2D4F0F0E2D102D8316DF02D9
:100A2000831250080318172D500F172D192D8316F8
:100A3000E00283165D088312CD0083165E088312E0
:100A4000CE0083165F088312CF00831660088312DE
:100A5000D00083124D088316D90083124E088316E6
:100A6000DA0083124F088316DB00831250088316C6
:100A7000DC0008007E302C0203185B2DAC08031943
:100A8000422D4A2D83124D084E044F045004FF3965
:100A90000319512D01308316DD00DE01DF01E00175
:100AA000562D8316DD01DE01DF01E001D501D601FF
:100AB000D701D8019A2D8312CF174D088316DD0078
:100AC00083124E088316DE0083124F088316DF0060
:100AD000831250088316E0001F305205E100E10840
:100AE0000319792D0310DD0DDE0DDF0DE00DE1039F
:100AF0006F2D83124D088316D50083124E0883167E
:100B0000D60083124F088316D7008312500883162D
:100B1000D800D209D309D20A0319D30A5208E10036
:100B2000E10803199A2D580DD80CD70CD60CD50C0A
:100B3000E103902D5D085E045F046004FF39031D2E
:100B4000AB16AA08031DE22DE01FC32DD50A031919
:100B5000D60A0319D70A0319D80A5D08E1005E080E
:100B6000E2005F08E3006008E4000310E10DE20D1D
:100B7000E30DE40D6108620463046404FF39031D9E
:100B8000C32DFE30D505AE080319242E5508003CB0
:100B9000E1000030E200E300E4005608031C560FB9
:100BA000E2025708031C570FE3025808031C580FB2
:100BB000E4026108D5006208D6006308D700640823
:100BC000D800242EE1015D085E045F046004FF3953
:100BD000031D6114AE080319162E2A03031DFA2DF6
:100BE000E1080319FA2DD50A0319D60A0319D70A01
:100BF0000319D80A5508003CE2000030E300E40085
:100C0000E5005608031C560FE3025708031C570F54
:100C1000E4025808031C580FE5026208D500630877
:100C2000D6006408D7006508D800242E2A08023AA6
:100C3000031D242EE1080319242ED50A0319D60A10
:100C40000319D70A0319D80A5508D9005608DA003B
:100C50005708DB005808DC0008004A088312CD0062
:100C600083164B088312CE0083164C088312CF00E4
:100C7000CF13D00183164D08AC00AC130310AC0D9C
:100C8000CC1B2C144E088312D10083164F088312FC
:100C9000D200831650088312D300D313D4018316D5
:100CA0005108AD00AD130310AD0DD01B2D14AE01D6
:100CB000CD1F5C2E0130AE00AF01D11F612E01307F
:100CC000AF002F082E06B00052102C0A0319521440
:100CD000D2102D0A0319D214521183124D084E045A
:100CE0004F045004FF39031D772E831652158316C7
:100CF000D21183125108520453045404FF39031DC6
:100D0000832E8316D21583165218882ED21CCE2E0F
:100D1000521C902E5219902E4C1B902E2B14C02E2C
:100D2000D21C982ED219982E501B982E2B14C02E00
:100D3000521C9C2E521DC02ED21CA02ED21DC02E85
:100D4000D21DA72EAD08031DA72E2B14C02E521D99
:100D5000AE2EAC08031DAE2E2B14C02ED801D90127
:100D60007F30DB008030DA00B008031DDB175B0842
:100D7000DF005A08DE005908DD005808DC000800D2
:100D8000D801D901C030DA00FF30DB005B08DF009A
:100D90005A08DE000030DD00DC0008007F30D300A0
:100DA000AC08031DF12E521DE52ED801D901DB013F
:100DB000DA01B008031DDB175B08DF005A08DE000C
:100DC0005908DD005808DC000800D3038312CF1B4C
:100DD000F32E0310CD0DCE0DCF0DD00D8316D30AFB
:100DE000E62E8312CF178316AD08031D152FD21DD3
:100DF000092FD801D901DB01DA01B008031DDB1787
:100E00005B08DF005A08DE005908DD005808DC00E6
:100E10000800D3038312D31B172F0310D10DD20D5B
:100E2000D30DD40D8316D30A0A2F8312D31707309C
:100E30008316D800D8080319262F03108312CD0D6E
:100E4000CE0DCF0DD00D8316D8031A2F0830D80041
:100E5000D8080319342F03108312D10DD20DD30DEE
:100E6000D40D8316D803282F7921F4080319F50827
:100E70000319702F74098316D8007509D900D80A90
:100E80000319D90A2030580259080318492F0319A9
:100E90004B2FD91F632F52127409DA00DA0A83121A
:100EA000551C542F8316521603108312D80CD70CDE
:100EB000D60CD50C8316DA03031D4F2F521E702F4C
:100EC00083125514702F8312550856045704580482
:100ED000FF390319702F0130D500D601D701D80191
:100EE00083162C08F400F5012D08F4070318F50A01
:100EF0005308F402031CF5038312581B882F0310B8
:100F0000D50DD60DD70DD80DF4080319F503F4034C
:100F100023205D21831255088316D40083125608BE
:100F20008316D500831257088316D60083125808FB
:100F30008316D7005708DF005608DE005508DD008D
:100F40005408DC00080052088312D50083165308A9
:100F50008312D600831654088312D70083165508CF
:100F60008312D8005508003C031DCA2F5608003CC8
:100F7000031DCA2F5708003C031DCA2F5808803C88
:100F8000031DCA2F01308316B0009E30F400F50116
:100F90008A150E288316B00183128A15D81F0828D7
:100FA00001308316B00083125508003C8316DA0026
:100FB0000030DB00DC00DD00831256088A110318C4
:100FC000E42F560FE42FE62F8316DB028312570817
:100FD0000318ED2F570FED2FEF2F8316DC0283122E
:100FE00058080318F62F580FF62FF82F8316DD0236
:100FF00083165A088312D50083165B088312D60025
:1010000083165C088312D70083165D088312D8000C
:101010009C30F400F5018A11042323208A115D21FC
:10102000831255088316D600831256088316D700FC
:10103000831257088316D800831258088316D900E4
:101040005908DD005808DC005708DB005608DA00B4
:10105000080083160313A80183120C108F018E0160
:1010600081010B118B1610148B170800FD08031D4E
:101070006B280F3083160313CA000130CB008A118E
:10108000D2220F308316CA000230CB00D2220F309A
:101090008316CA000330CB00D2220F308316CA0059
:1010A0000430CB00D2220F308316CA000530CB00AB
:1010B000D2228316CA010630CB00D2228316CA017F
:1010C0000730CB00D2220B308316CA000830CB0089
:1010D000D2228A15F428831203130F08E400E501D5
:1010E0000F08E600E70166086406031D7B28670811
:1010F000650603197E280F08E400E5018316B20196
:10110000831264088316B30032088312EA00831640
:1011100033088312EB000E086A048316B2008312B0
:101120006B088316B30032088312E8008316330875
:101130008312E900033062028316B600831263084B
:101140008316B700031CB7033608B2003708B30094
:101150000330B400B5018A1178223F08B800400876
:10116000B9003808283EBA003908BB000318BB0A8A
:101170003A088312EC0083163B088312ED000E3010
:1011800068028316B200B030031CB13083126902CA
:101190008316B30000303207B4003308B500803046
:1011A0000318B50AB5078312600883163407B60022
:1011B000831261088316B70035080318B70AB7070A
:1011C00083126C0883163607B80083126D088316E5
:1011D000B90037080318B90AB90738088312E800BC
:1011E000831639088312E9007D08013CFE000800DF
:1011F000831205108316B8012030380203184829DD
:101200003808B900BA01BB01BC013A083B043C04F0
:10121000FF3903191029BD01BE01BF01C0012B29EF
:101220003208C5003308C6003408C7003508C800B6
:101230003908C900031923290310C80CC70CC60CB0
:10124000C50CC9031A294508BD004608BE00470859
:10125000BF004808C00001303D05C10000303E0518
:10126000C20000303F05C30000304005C400410803
:10127000420443044404FF390319412983128514AD
:10128000432983128510051505118316B80AFC2819
:10129000B80108303802031872293608BD00370833
:1012A000BE003808BF0003195A29370DBE0CBD0C0B
:1012B000BF0353293D08B9003E08BA000130390583
:1012C000BB00BC01BB08031D6829BC0803196B29BE
:1012D000831285146D298312851005150511831657
:1012E000B80A492983120514051008008312031354
:1012F000901210129011101590148F018E01080099
:1013000083160313811781128111011581140114B1
:101310000B118B128B130800FB08031DA72901304A
:1013200083160313A300831205128316A408031D5A
:10133000A72983126808F2006908F30001308316B8
:10134000A4000D30CA000830CB008A11D2228312CB
:10135000031327088316B2000130B3003208CA0015
:101360003308CB008A11D22283128A158619F529F7
:101370008316A101A20183120619D9298316A10897
:10138000031DB42983123D088316B20083123E0860
:101390008316B30083123F088316B40083124008FB
:1013A0008316B500B601B701F82001308316A100FD
:1013B000B4298316A208031DB42983123D0883169D
:1013C000B20083123E088316B30083123F088316CF
:1013D000B400831240088316B5000430B600B7018C
:1013E000F82001308316A200B429061908003D0830
:1013F0008316B20083123E088316B30083123F089F
:101400008316B400831240088316B5000430B6007A
:10141000B701F82001308316A200080008308312BB
:1014200003130605F70080300605F90008300605AD
:101430008316B20077083206031D2B2A7808770638
:1014400003192B2A7708F800F70803192A2A013014
:10145000F6002B2AF6018030831206058316B300AE
:1014600079083306031D552A7A0879060319552A87
:10147000F908031D4B2A0A30B4008A1110200130EC
:10148000FB0096308312EE00EF01831601138B10E0
:101490000B168A15532A3230B4008A111020FB0132
:1014A0008B100B128B137908FA008312E201E3010F
:1014B0008A1506185E2A0130E200E301061A712A35
:1014C000023062078316B400831263088316B500E6
:1014D0000318B50A34088312E20083163508831214
:1014E000E300861A0800043062078316B4008312F2
:1014F00063088316B5000318B50A34088312E200A6
:10150000831635088312E300080083120313851540
:1015100005118510FF308316CA000930CB008A11EF
:10152000D22207308316CA000B30CB00D222013002
:101530008316CA000C30CB00D2228316CA010F30AA
:10154000CB00D2220800FB08031DEF2A83160313E9
:10155000A8080319AE2A36208A1529208316A40864
:101560000319ED2A3D307202B2007308B300031C68
:10157000B3038312690883163302031DC32A83123F
:101580006808831632020318D72A3D307207B40068
:101590007308B5000318B50A350883126902031DE4
:1015A000D52A8316340883126802031C112B0330DA
:1015B000831625020318DF2A250AA500112BA50191
:1015C000A301831205168316A4010F30CA00083048
:1015D000CB008A11D2228A15112BA501112B83125F
:1015E00003136E08003E8316B20083126F08831641
:1015F000B30080300318B30AB30732088312E8003F
:10160000831633088312E9008316A501A301831210
:1016100005168316A4010F30CA000830CB008A11CA
:10162000D222FE088A15031DDC2C8316A408031D94
:101630009E2C83126908803C031D202B6808003C07
:10164000031C392B4508BD004608BE004708BF00F3
:101650004808C0000D308316CA000130CB008A1143
:10166000D2228316CA010630CB00D2220130831663
:10167000A600A730831269028A15031D412B103082
:101680006802031C5B2B4908BD004A08BE004B08DA
:10169000BF004C08C0000C308316CA000130CB00DC
:1016A0008A11D22202308316CA000630CB00D22221
:1016B00001308316A6008316A6088A15031D7D2C0B
:1016C000831268088316B600831269088316B70070
:1016D000B801B9013608BA003F303705BB00003009
:1016E0003805BC0000303905BD003A08B2003B089F
:1016F000B3003C08B4003D08B500CA01CB01A030DE
:10170000CC004130CD003208D2003308D300340879
:10171000D4003508D5008A11A3275A08CE005B08EB
:10172000CF005C08D0005D08D1002D265C08BE000B
:101730005D08BF005E08C0005F08C1003E08CE0023
:101740003F08CF004008D0004108D1007F2459084D
:10175000C2005A08C3005B08C4005C08C500003022
:10176000D7002030CA005708CB002530CE003030DB
:10177000CF003830D0007530D100D2010030D70012
:10178000CE30CC005708CD004208D3004308D40027
:101790004408D5004508D6001C230F30CA0001308C
:1017A000CB00D22226088316CC000230CD004C0894
:1017B000CA004D08CB00D22225088316CC00033086
:1017C000CD004C08CA004D08CB00D2228030240442
:1017D0008316CC000430CD004C08CA004D08CB0065
:1017E000D22223088316CC000530CD004C08CA0055
:1017F0004D08CB00D22222088316CC000630CD0043
:101800004C08CA004D08CB00D22287308316CA008C
:101810000730CB00D2220F308316CA000830CB002D
:10182000D22239088316CA0083123A088316CB00E5
:1018300083123B088316CC0083123C088316CD002C
:101840003208D2003308D3003408D4003508D5005C
:10185000A3275A08CE005B08CF005C08D0005D08C3
:10186000D1002D265C08C6005D08C7005E08C800D0
:101870005F08C9004608CE004708CF004808D000DE
:101880004908D1007F245908831235078316CA00FE
:101890005A08CB00831236088A15031C522C360FC7
:1018A000522C542C8316CB0783165B08CC00831272
:1018B0003708031C5E2C370F5E2C602C8316CC0778
:1018C00083165C08CD0083123808031C6A2C380F7D
:1018D0006A2C6C2C8316CD0783164A088312BD0030
:1018E00083164B088312BE0083164C088312BF0078
:1018F00083164D088312C0009E2CCA010230CB0013
:101900008A11D2228316CA010330CB00D222803042
:101910008316CA000430CB00D2228316CA010530D8
:10192000CB00D22287308316CA000730CB00D222E8
:101930000B308316CA000830CB00D22283128A15DE
:10194000851EBB2CFC08031DA62CDC2C3D08831631
:10195000B20083123E088316B30083123F08831639
:10196000B400831240088316B5000430B600B701F6
:10197000F820FC01DC2C3D088316B20083123E08DF
:101980008316B30083123F088316B4008312400805
:101990008316B500B601B701F8200130FC008316AC
:1019A000A501A301831205168316A4010F30CA00F6
:1019B0000830CB008A11D2227B08013C7E058316B9
:1019C000B20026083204A700A601080007308312DF
:1019D00003139F00E0308316850083128501FF30DA
:1019E00083168600831286010800831203130511F3
:1019F0000510851005150511051405100800E624CD
:101A0000F001F10185228A15F524802176218B10C1
:101A10000B12861F0D2DFA010F2D0130FA000A302E
:101A20008316B4008A1110208A1529200E227B0803
:101A3000013C7E05FE00F608031DA322F6088A1568
:101A4000031D162D8316A708031D162D8C21162D98
:101A500083120313A901AA015030AB00AC01A530D9
:101A6000E000E101E103C030AD00CF30AE006A30EC
:101A7000AF00B001B101B201A030B3004130B400F9
:101A80003330B500E130B6005530B7000E30B80045
:101A9000D430B900CA30BA002B30BB004430BC008F
:101AA0000130F600F701F801F901FA01FB01E2014A
:101AB000E301FC01FD01FE0132308316A000643019
:101AC0008312EE00EF01C101C201C301C401350858
:101AD000C5003608C6003708C7003808C800C0303F
:101AE000C900BB30CA00BE30CB000E30CC0083161C
:101AF000A101A201A301A401A501A601A701A801BA
:101B00008312CD01CE01CF01D001D101D201D30189
:101B1000D401D501D601D701D8018316AC01AD019E
:101B2000F401F501AE01AF01B001B1018312D90199
:101B3000DA01DB01DC018316AA01AB01A9018A15D8
:101B40000A12FF2C0B1DAF2D8B13831203131010E1
:101B50008B1201300C05FD0001308316A8008312A2
:101B60000313861B582E8B1C582E0618072E061E94
:101B7000DF2D861ECD2D6E080317A50003136F08F9
:101B80000317A600A50A0319A60A25080313EE00E9
:101B9000031726080313EF00042E0A306E070317FD
:101BA000A50003136F080317A6000318A60A25084B
:101BB0000313EE00031726080313EF00042E861EFE
:101BC000F32D01306E020317A50003136F080317EE
:101BD000A600031CA60325080313EE00031726081E
:101BE0000313EF00042E0A306E020317A50003133F
:101BF0006F080317A600031CA60325080313EE00B5
:101C0000031726080313EF0083160117562E061E2E
:101C10002F2E861E1D2E01306E020317A500031302
:101C20006F080317A600031CA60325080313EE0084
:101C3000031726080313EF00542E0A306E02031711
:101C4000A50003136F080317A600031CA6032508AD
:101C50000313EE00031726080313EF00542E861E0D
:101C6000432E6E080317A50003136F080317A60081
:101C7000A50A0319A60A25080313EE000317260870
:101C80000313EF00542E0A306E070317A500031349
:101C90006F080317A6000318A60A25080313EE0011
:101CA000031726080313EF00831601138B108B17FD
:101CB00083125F0E84005E0E8A005D0E8300FF0EAD
:041CC0007F0E09008A
:02400E00013F70
:00000001FF
